:020000040800F2
:1000000000040020E1010008E3010008E30100080A
:10001000E3010008E3010008E3010008E301000830
:10002000E3010008E3010008E3010008952E000841
:10003000E3010008E3010008E3010008E301000810
:10004000E3010008E3010008E3010008E301000800
:10005000E3010008E3010008F93000082531000839
:10006000513100087D310008A9310008E301000882
:10007000E3010008E3010008E3010008E3010008D0
:10008000E3010008E3010008E3010008E3010008C0
:10009000E3010008E3010008E3010008D53100088E
:1000A000E3010008E3010008E3010008E3010008A0
:1000B000E3010008E3010008E3010008E301000890
:1000C000E3010008E3010008E3010008E301000880
:1000D000E3010008E3010008E3010008E301000870
:1000E0003D320008E3010008E3010008E3010008D5
:1000F000E3010008E3010008E3010008E301000850
:10010000E3010008E3010008112F0008E3010008E3
:10011000E3010008E3010008E3010008E30100082F
:10012000E3010008E3010008E3010008E30100081F
:10013000E3010008E3010008E3010008E30100080F
:10014000E3010008E3010008E3010008DD250008E1
:10015000E3010008E3010008E3010008E3010008EF
:10016000E3010008E3010008E3010008E3010008DF
:10017000E3010008E3010008E3010008E3010008CF
:10018000E3010008E3010008E3010008E3010008BF
:10019000E3010008E3010008E3010008E3010008AF
:1001A000E3010008E3010008E3010008E30100089F
:1001B000E3010008E3010008E3010008E30100088F
:1001C000E3010008E3010008E3010008E30100087F
:1001D000E3010008E3010008E3010008E30100086F
:1001E00002E000F000F8FEE772B6394880F30888B4
:1001F000384880F3098838484EF60851CEF200019D
:10020000086040F20000CCF200004EF63471CEF2ED
:1002100000010860BFF34F8FBFF36F8F40F2000003
:10022000C0F2F0004EF68851CEF200010860BFF334
:100230004F8FBFF36F8F4FF00000E1EE100A4EF6C4
:100240003C71CEF200010860062080F31488BFF3F1
:100250006F8F01F08BFE02F0B3FD4FF055301F4958
:100260001B4A91423CBF41F8040BFAE71C49194A6A
:1002700091423CBF41F8040BFAE71A491A4A1B4B5A
:100280009A423EBF51F8040B42F8040BF8E70020F5
:100290001749184A91423CBF41F8040BFAE701F0B4
:1002A00069FE02F0E9FD144C144DAC4203DA54F837
:1002B000041B8847F9E700F03FF8114C114DAC42A0
:1002C00003DA54F8041B8847F9E701F051BE000037
:1002D000000400200024002000000008000000208E
:1002E000000400207036000800240020282400208C
:1002F0002824002038340020E0010008E001000834
:10030000E0010008E00100082DE9F04F2DED108A12
:10031000C1F80CD0C3689D46BDEC108ABDE8F08FD3
:10032000002383F311882846A047002001F0C4FA77
:1003300001F074FA00DFFEE71B4B7F2270B51A70E4
:1003400004225A706FF03F0200245A720F229C70F0
:10035000DC701C715C719C71DC711C729A72DC72B5
:1003600001F0DAFD064601F0FBFD054650B90F4BE2
:100370009E4217D001339E4241F2883412BF054697
:1003800000240125002001F0CDFD0DB100F0B4F8EE
:1003900000F038FD00F002FC204600F00BF900F000
:1003A000ABF8F9E70446EDE728240020010007B088
:1003B00008B500F095FBA0F120035842584108BD54
:1003C00007B5054B02211B88ADF8043001A800F0E9
:1003D000D5FB03B05DF804FB38330008064991F8FB
:1003E000243033B100230822086A81F8243000F059
:1003F000F7BB0120704700BF482400202DE9F84FCB
:10040000234C94F824300546884617468BBB2E466D
:10041000DFF87C90002F38D094F824A0BAF1000FB8
:1004200005D12022FF214846266200F0D9FCCAF1FE
:100430000805BD4228BF3D465FFA85FBAD00414639
:100440002A4604EB8A0000F0A1FC94F82430A7EBC4
:100450000B079B445FFA8BFBBBF1080F2E44A844AB
:10046000FFB284F824B0D5D1FFF7B8FF0028D1D16E
:1004700008E0266A06EB8306B042C9D0FFF7AEFF5C
:100480000028C4D10020BDE8F88F0120BDE8F88F16
:100490004824002010B5202383F311881248C36834
:1004A0000BB101F08FFA0023104A0F484FF47A7114
:1004B00001F04CFA002383F311880D4C236813B12B
:1004C0002368013B2360636813B16368013B636089
:1004D000084B1B7833B9636823B9022000F042FC53
:1004E0003223636010BD00BF34240020950400084F
:1004F000782900207024002010B5254B254953F899
:10050000042F013200D110BD8B42F8D1224C234B75
:1005100022689A423AD9224B9B6803F1006303F5A3
:1005200080439A4232D2002000F052FB1D4B022041
:10053000187000F007FC1C4B1A6C00221A64196E2C
:100540001A66196E596C5A64596E5A665A6E5A690F
:1005500042F080025A615A6922F080025A615A6957
:100560001A6942F000521A611A6922F000521A61A7
:100570001B6972B60D4A0E4B13601B68226820215E
:1005800081F311889D4683F30888104710BD00BF92
:10059000FC3F00081C40000804400008FF3F000822
:1005A00028240020702400200038024008ED00E0DC
:1005B000004000082DE9F04FB04C97B02022814652
:1005C000FF210EA8A66800F00BFCAD4A1378A346E5
:1005D000A3B9AC480121C3601170202383F31188B3
:1005E000C3680BB101F0EEF90023A74AA5484FF408
:1005F0007A7101F0ABF9002383F31188B9F1000F90
:1006000002D0A24BC3F80090A14BA04A00241C705A
:100610005460254627469846012000F093FBB9F127
:10062000000F00F02282994B1B68002B40F01D82C6
:1006300017B0BDE8F08F0220FFF7BAFE002840F0A7
:100640000E82944B1B88ADF82430022109A800F0DB
:1006500095FAE1E74FF47A7000F042FA031E019335
:10066000EFDB0220FFF7A4FE82460028E9D0019BC1
:10067000581E042800F2F581DFE800F0030D101386
:10068000160016A8052340F8343D042100F076FA40
:100690005446002752E004217848F7E704217E48B9
:1006A000F4E704217D48F1E71C24204600F092FA8B
:1006B00004340990042109A800F060FA2C2CF4D12C
:1006C000E6E7002DBDD0002CBBD00220FFF770FE66
:1006D0000546002800F0C781012000F079FA0220C9
:1006E00088F8000000F02EFB0024E3B218460193C6
:1006F00000F07EFA824648B1019B184600F088FA65
:1007000001340028F1D12C46654B9BE701230220E0
:1007100088F8003000F004FB5646DBF808309E42B3
:1007200006D2304600F056FA0130ECD10436F4E738
:10073000564B002688F800605E602C4600F058FB9F
:100740001DB1002C18BF4FF00009FFF739FE63E719
:10075000002D3FF476AF002C3FF473AF022088F8F1
:10076000000000F0EFFA322000F0BAF9B0F1000A10
:10077000C0F279811AF0030540F07581DBF808209A
:1007800006EB0A03934200F26E81BAF5807F00F215
:100790006A81444B019355450DDA4FF47A7000F0AD
:1007A0009FF90290029A002AC0F25D81019B029A91
:1007B000EA540135EEE7C820FFF7FAFD05460028A8
:1007C00000F051811F2E11D8C6F12004544528BFD6
:1007D00054460EAB26F0030022463249184400F07E
:1007E000D5FA2246FF212F4800F0FAFA4FEAAA0A6A
:1007F0005FFA8AF22B493046FFF700FE04460028D4
:1008000081D006EB8A06054698E70220FFF7D0FD67
:1008100000283FF416AFFFF7E1FD00283FF411AFC9
:1008200000229246DBF808309A4259D21F2A1ED87D
:100830000E9B01331BD022F0030316A90B4453F87F
:10084000203C09931848436883B3174800210DF1F1
:10085000240E11F80E3083EA0A03DBB2013150F89E
:100860002330042983EA1A2AF3D10432DAE7104646
:10087000019200F0AFF9019A0990E3E728240020E3
:1008800074250020342400209504000878290020D5
:10089000702400203A3300082C240020302400204B
:1008A0003C330008742400207825002019464FF0BE
:1008B000080E11F0010F4FEA51011FBF81F06D4189
:1008C00081F4380181F4034181F02001BEF1010E71
:1008D000EFD140F823100133B3F5807FE6D1B4E7C0
:1008E00016A8042140F84CAD00F048F926E716A8F8
:1008F000002340F8343D642100F01CF900287FF407
:10090000A0AE0220FFF754FD00283FF49AAE0998EC
:1009100000F090F916AB43F8480D04211846E3E7C0
:1009200016A8002340F8343D642100F003F90028A4
:100930007FF487AE0220FFF73BFD00283FF481AE35
:10094000099800F085F916AB43F8440DE5E702205D
:10095000FFF72EFD00283FF474AE00F07FF916ABD0
:1009600043F8400DD9E70220FFF722FD00283FF4AD
:1009700068AE09A9142000F077F9824616A8042170
:1009800040F83CAD00F0FAF8514609A8ACE7322037
:1009900000F0A6F8B0F1000AFFF653AE1AF0030F0C
:1009A0007FF44FAEDBF808200AEB070393423FF6D3
:1009B00048AE0220FFF7FCFC00283FF442AE2AF0CC
:1009C000030ABA44BA453FF4B9AE384600F002F91A
:1009D0000421089008A800F0D1F80437F2E74FF49A
:1009E0007A70FFF7E5FC00283FF42BAEFFF7F6FC2A
:1009F00000283FF489AE0E9B01330CD008220EA9CB
:100A00000020FFF7FBFC00283FF47EAE2022FF21F0
:100A10000EA800F0E5F9FFF7D3FC304800F052FFD4
:100A200006E616A8002340F8343D642100F082F861
:100A3000824600287FF405AE0220FFF7B9FC0028AB
:100A40003FF4FFADFFF7BCFC41F2883000F03AFF05
:100A5000099800F001FAD14600F0CAF9DCE5054634
:100A60006CE60027EDE52546EBE5002000F038F8C0
:100A70000290029B002BFFF6D2AD012000F050F94E
:100A8000029B213B122B3FF6C7AD01A252F823F087
:100A90003706000855060008C306000819060008B6
:100AA0001906000819060008510700088F090008F8
:100AB0000B080008EF080008210900084F0900088A
:100AC000190600086709000819060008DF09000870
:100AD0003D07000819060008230A0008A086010047
:100AE00037B5114B1A780132D2B20024012A0146DF
:100AF0008DF8074011D80D4803681D6A4FF47A73CA
:100B00004B4301220DF10701A847012805D1084BED
:100B10009DF807001C7003B030BD4FF4FA7000F070
:100B2000D1FE4FF0FF30F6E700240020C829002056
:100B30008429002038B50E4B1A780132D2B2012A2E
:100B400005460ED80B4803681C6A4FF47A734B4372
:100B500004222946A047042803D1074B002018701F
:100B600038BD4FF4FA7000F0ADFE4FF0FF3038BDE5
:100B700000240020C82900208429002030B4054C1E
:100B80002368DD69044B0A46AC460146204630BC6A
:100B9000604700BFC8290020A086010070B501F0A1
:100BA000DBF8094C094E2070002530682378834219
:100BB00008D901F0CBF8336805440133B5F5804F0F
:100BC0003360F2D370BD00BF85290020802900204A
:100BD00001F06CB900F1006000F5804000687047DA
:100BE00000F10060920000F5804001F0F7B80000CD
:100BF000054B1A68054B1B789B1A834202D9104497
:100C000001F0A4B800207047802900208529002029
:100C100038B5074D04462868204401F09FF828B9EC
:100C200028682044BDE8384001F0B0B838BD00BFA6
:100C30008029002010F0030308D1B0F5007F05D80B
:100C400000F10050A0F50840006870470020704790
:100C5000014BC058704700BF107AFF1F014B186846
:100C6000704700BF002004E070B52A4B1C68C4F335
:100C70000B03240C63B140F21342934231D040F293
:100C8000194293422FD040F2214293422DD10323A7
:100C9000214A0C2505FB03235D6893F9082042F2E5
:100CA00001039C4224D0B4F5805F23D041F20103BC
:100CB0009C4221D041F203039C421FD041F2070322
:100CC0009C4208BF3122441E0C44013D0B46A34206
:100CD0001ED215F9016F581C96B1034600F8016C3D
:100CE000F5E70123D4E70223D2E73F220B4DD6E7F5
:100CF0003322E3E74122E1E75A22E4E75922E2E71F
:100D00002C2584421D7001D9981C5A70401A70BD60
:100D10001846FBE7002004E04C330008403300088D
:100D2000022804D1054B4FF080429A617047012898
:100D3000FCD14FF40012024BF7E700BF000C024059
:100D400000080240022804D1044B4FF480429A610B
:100D500070470128FCD12022014BF8E7000C02402B
:100D600000080240022805D1064A536983F48043F3
:100D7000536170470128FCD1034A536983F0200373
:100D8000F6E700BF000C02400008024010B5002347
:100D9000934203D0CC5CC4540133F9E710BD00008A
:100DA00030B5441E14F9010F0B4660B193F90050A1
:100DB000854201F1010106D11AB993F90020801A88
:100DC00030BD013AEEE7002AF7D1104630BD0000F1
:100DD00002460346981A13F9011B0029FAD17047FD
:100DE00002440346934202D003F8011BFAE770471E
:100DF000024B1A78024B1A70704700BF84290020FA
:100E00000024002038B5104D104C284600F0A2F800
:100E10002146284600F0CAF823680D485A6DD2F8DA
:100E2000043843F00203C2F8043800F04BFD0949CE
:100E3000206800F0C7F923685A6DD2F8043823F00F
:100E40000203C2F8043838BDC8290020183400084D
:100E500040420F006C34000870470000026843688D
:100E60001143016003B118477047000013B5446B8C
:100E7000D4F894341A681178042915D1217C0229F8
:100E800012D11979128901238B4013420CD101A987
:100E900004F14C0001F008FED4F89444019B217940
:100EA0000246206800F0DAF902B010BD143001F0FB
:100EB0008BBD00004FF0FF33143001F085BD000002
:100EC0004C3001F05DBE00004FF0FF334C3001F0BC
:100ED00057BE0000143001F059BD00004FF0FF3143
:100EE000143001F053BD00004C3001F029BE000069
:100EF0004FF0FF324C3001F023BE0000D0F89424B4
:100F000038B5136819780429054601D0012038BD89
:100F1000017C0229FAD112795C89012090400440B9
:100F2000F4D105F1140001F0EBFC02460028EDD0ED
:100F3000D5F894544FF480732868697900F07CF9EF
:100F4000204638BD406BFFF7D9BF00000020704736
:100F5000704700007FB5124B03600023436083603D
:100F6000C360012502260F4B0574044602900193CD
:100F700000F18402294600964FF48073143001F08A
:100F80009BFC094B0193029400964FF4807304F587
:100F90002372294604F14C0001F062FD04B070BDDB
:100FA0009C330008450F00086D0E00080B682022D6
:100FB00082F311880A7903EB820290614A7909323F
:100FC00043F822008A7912B103EB8203986102236D
:100FD0000374C0F89414002383F311887047000051
:100FE00038B5037F044613B190F85430ABB9201DD7
:100FF00001250221FFF732FF04F1140025776FF07D
:10100000010100F087FC84F8545004F14C006FF0AB
:101010000101BDE8384000F07DBC38BD10B50121AC
:1010200004460430FFF71AFF0023237784F8543076
:1010300010BD000038B504460025143001F054FC02
:1010400004F14C00257701F023FD201D84F8545055
:101050000121FFF703FF2046BDE83840FFF74EBFF0
:1010600090F8443003F06003202B19D190F845200C
:10107000212A0AD0222A4FF000030ED0202A0FD1B5
:10108000084A82630722C26304E0064B8363072396
:10109000C36300230364012070478363C363F9E7DC
:1010A0000020704701240020D0F8943437B51A6826
:1010B0001178042904461AD1017C022917D1197923
:1010C000128901238B40134211D100F14C052846AF
:1010D00001F09EFD58B101A9284601F0E5FCD4F8C5
:1010E0009444019B21790246206800F0B7F803B0D0
:1010F00030BD000000EB8103F7B59C6905460E4644
:10110000F4B1202383F3118805EB8607201D082105
:10111000FFF7A4FEFB685B691B684C3413B12046E3
:1011200001F0D0FC01A9204601F0BEFC024648B106
:10113000019B3146284600F091F8002383F3118883
:1011400003B0F0BDFB685A691268002AF5D01B8A0B
:10115000013B1340F1D105F14402EAE7093138B50A
:1011600050F82140DCB1202383F31188D4F8942473
:101170001368527903EB8203DB689B695D6845B1B4
:1011800004216018FFF76AFE294604F1140001F0FB
:10119000C1FB2046FFF7B2FE002383F3118838BD60
:1011A0007047000000F06CBF012303700023436010
:1011B000C36183620362C362436203630381438149
:1011C0007047000038B50446202383F311880025BA
:1011D0004160C56005614561856100F061FF0223E2
:1011E000237085F3118838BD70B500EB8103054687
:1011F0005069DA600E46144618B110220021FFF73C
:10120000EFFDA06918B110220021FFF7E9FD31467A
:101210002846BDE8704001F00DB80000028902F0D8
:1012200001020281428902F0010242810022026130
:101230004261826101F092B8F0B400EB8104478909
:10124000E4680125A4698D403D4345812360002366
:10125000A2606360F0BC01F0ADB80000F0B400EB38
:1012600081040789E468012564698D403D43058157
:1012700023600023A2606360F0BC01F027B9000086
:1012800070B50223002504460370A0F84C5080F886
:101290004E5080F84F5005814581C560056145611C
:1012A000856180F8345000F061FF63681B6823B1EA
:1012B00029462046BDE87040184770BD4368027853
:1012C0001B6880F85020052202700BB104211847DA
:1012D00070470000436890F850201B6802700BB103
:1012E000052118477047000090F8343070B5044667
:1012F00013B1002380F8343004F14402204601F099
:101300004FF863689B6863BB94F8445015F060061F
:1013100015D194F8453005F07F0545EA032540F2E4
:1013200002339D4200F00E815BD8022D00F0DC807C
:101330003FD8002D00F08780012D00F0CF800021E4
:10134000204601F085FA0021204601F077FA636813
:101350001B6813B1062120469847062384F83430D1
:1013600070BD204698470028CED094F84B2094F8C2
:101370004A3043EA0223E26B934238BFE36394F9B5
:101380004430E56B002B4FF0200380F2FD80002DF0
:1013900000F0EC80092284F8342083F311880021C6
:1013A000E36BA26B2046FFF759FF002383F31188FC
:1013B00070BDB5F5817F00F0B180B5F5407F49D0B3
:1013C000B5F5807FBBD194F84630012BB7D1B4F886
:1013D0004C3023F00203A4F84C30A663E663266485
:1013E000C3E740F201639D421ED8B5F5C06F3BD202
:1013F000B5F5A06FA3D1B4F84430B3F5A06F0ED10A
:1014000094F8463084F84E30204600F007FF6368B9
:101410001B6813B101212046984703232370002342
:10142000A363E3632364A0E7B5F5106F32D040F601
:1014300002439D4252D0B5F5006F80D104F14F03B5
:10144000A363012324E004F14C03A3630223E363B9
:1014500025648AE794F84630012B7FF470AFB4F826
:101460004C3043F00203B6E794F84920616894F8E1
:1014700048304D6894F8471043EA0223204694F818
:101480004620A84700283FF45AAF4368A363036887
:10149000E363A4E72378042B10D1202383F311887E
:1014A0002046FFF7BBFE86F31188636884F84F601F
:1014B0001B68032121700BB12046984794F84630F1
:1014C000002BACD084F84F300423237063681B6872
:1014D000002BA4D0022120469847A0E7374BA363F6
:1014E0000223E36300239DE794F8481011F0800F76
:1014F000204601F00F010ED000F044FF012806D075
:1015000002287FF41CAF2E4BA363E06367E72D4BEB
:10151000A363E56363E700F027FFEFE794F8463045
:10152000002B7FF40CAF94F8483013F00F013FF418
:1015300076AF1A06204602D501F09EF96FE701F05A
:1015400091F96CE794F84630002B7FF4F8AE94F8EC
:10155000483013F00F013FF462AF1B06204602D55E
:1015600001F076F95BE701F069F958E7142284F895
:10157000342083F311882B462A4629462046FFF75C
:101580005BFE85F3118870BD5DB1152284F83420AF
:1015900083F311880021E36BA26B2046FFF74CFE1A
:1015A00003E70B2284F8342083F311882B462A4664
:1015B00029462046FFF752FEE3E700BFCC33000880
:1015C000C4330008C833000838B590F834300446F6
:1015D000152B29D8DFE803F03E28282828283E28A4
:1015E000280B293928282828282828283E3E90F822
:1015F0004B1090F84A20C36B42EA01229A4214D958
:10160000C268128AB3FBF2F502FB15356DB92023CF
:1016100083F311882B462A462946FFF71FFE85F3E0
:1016200011880A2384F8343038BD142384F8343008
:10163000202383F3118800231A4619462046FFF71A
:10164000FBFD002383F3118838BD036C03B1984779
:101650000023E7E7002101F0FBF80021204601F01C
:10166000EDF863681B6813B10621204698470623EE
:10167000D8E7000090F83420152A38B5044622D85F
:101680000123934040F6416213421DD113F48015AB
:101690000FD19B0217D50B2380F83430202383F31E
:1016A00011882B462A462946FFF7D8FD85F3118875
:1016B00038BDC3689B695B682BB9036C03B198475D
:1016C000002384F8343038BD002101F0C1F8002136
:1016D000204601F0B3F863681B6813B10621204669
:1016E00098470623EDE70000024B00221B605B6079
:1016F0009A60704788290020002303748268054B94
:101700001B6899689142FBD25A680360426010607E
:10171000586070478829002008B5202383F311887A
:10172000037C032B05D0042B0DD02BB983F3118838
:1017300008BD436900221A604FF0FF334361FFF791
:10174000DBFF0023F2E790E80C001A6002685360A8
:10175000F2E70000002303748268054B1B68996858
:101760009142FBD85A68036042601060586070472D
:1017700088290020054B19690874186802681A60E6
:101780005360186101230374FEF7BEBD8829002051
:1017900030B54B1C87B005460A4C10D023690A4A65
:1017A00001A800F0D3F82846FFF7E4FF049B13B12B
:1017B00001A800F007F92369586907B030BDFFF7A9
:1017C000D9FFF8E7882900201917000838B50C4D13
:1017D00041612B6981689A689142044603D8BDE84B
:1017E0003840FFF789BF1846FFF786FF01232C61B9
:1017F000014623742046BDE83840FEF785BD00BF92
:1018000088290020044B1A681B6990689B689842DD
:1018100094BF0020012070478829002010B5084C93
:10182000236820691A6822605460012223611A74B7
:10183000FFF790FF01462069BDE81040FEF764BD48
:1018400088290020826002220274002242747047BC
:101850008368A3F17C0243F80C2C026943F83C2C0A
:10186000426943F8382C074A43F81C2CC26843F8F5
:10187000102C022203F8082C002203F8072CA3F1F5
:10188000180070472103000810B5202383F3118846
:10189000FFF7DEFF00210446FFF798FF002383F3E4
:1018A0001188204610BD0000024B1B6958610F20B3
:1018B000FFF760BF88290020202383F31188FFF7FA
:1018C000F3BF000008B50146202383F311880820E8
:1018D000FFF75EFF002383F3118808BD49B1064B73
:1018E00042681B6918605A60136043600420FFF768
:1018F0004FBF4FF0FF30704788290020036898429F
:1019000006D01A680260506059611846FFF7F4BEAD
:101910007047000038B504460D462068844200D167
:1019200038BD036823605C604561FFF7E5FEF4E7BE
:10193000054B03F114025A619A614FF0FF32DA61EC
:1019400000221A62704700BF88290020F8B50361A1
:101950001A4BC2605C6A1A4B1A46022952F8145F8D
:1019600038BF0221954206461F460AD15861986148
:101970001C620560456081600819BDE8F84001F00F
:1019800069B9186AAB68241A0C1902D3E41A2D68D5
:1019900004E09C4202D2204401F06CF9AB689C4206
:1019A000F4D86B68736035601E606E60B460A968BF
:1019B0004FF0FF33091BA960FB61F8BD000C00402C
:1019C0008829002010B41A4C234653F8141F814272
:1019D00010D0416802680A60026851609A424FF074
:1019E0000001C16003D0936881680B4493605DF887
:1019F000044B70470A68626100209A425360C860D5
:101A000003D15DF8044B01F02FB993688868034453
:101A10009360084A206A526A121A9342E7D9991AC7
:101A2000012998BF931C18445DF8044B01F022B9BA
:101A300088290020000C004000207047FEE70000CD
:101A4000704700004FF0FF3070470000022906D0B9
:101A5000032906D00129064818BF00207047054811
:101A60007047032A9ABF044800EBC2000020704769
:101A7000C83400087C3400080824002070B50446EF
:101A800008460D46FFF7A4F9C6B220460134037894
:101A90000BB9184670BD32462946FFF781F9002878
:101AA000F3D1012070BD00002DE9F04F81469BB0BD
:101AB00008460D461646FFF78BF93D49C4B2284645
:101AC000FFF7DCFF08B10434E4B23A492846FFF7D7
:101AD000D5FF08B11034E4B2632C01AF0CD8DFF8A5
:101AE000E0A0DFF8E0B03C4695F80080B8F1000FC8
:101AF0001CD184F8008003E02946384601F014FC2C
:101B00003846FFF765F9C0B2431C5B0089E848001E
:101B1000337003237370002302361946DAB2904201
:101B200006F102063DD81BB0BDE8F08FB8F1250FD5
:101B300032D107221E492846FFF732F970B9DBF887
:101B400000202260DBF804206260BBF808202281BC
:101B50009BF80A20A27207350B34C5E70822154905
:101B60002846FFF71DF9B8B91348A21C10F8011F49
:101B7000124B4FEA111E01F00F011EF80AE011F896
:101B80000A1002F802EC984202F8011C02F102026B
:101B9000ECD118340835A7E784F80080013501340A
:101BA000A2E7FA5C06F8022C06F8011C0133B5E73F
:101BB00020340008283400080F7AFF1F1B7AFF1F0B
:101BC0003D3400083134000808B5202383F3118820
:101BD0000348FFF769FA002383F3118808BD00BFAB
:101BE000C829002010B50446052916D8DFE801F001
:101BF00016150316161D202383F311880E4A0121A2
:101C0000FFF7F2FA20460D4A0221FFF7EDFA0C48E1
:101C1000FFF710FA002383F3118810BD202383F30C
:101C200011880748FFF7DCF9F4E7202383F31188D4
:101C30000348FFF7F3F9EDE7D0330008F433000869
:101C4000C829002038B50C4D0C4C0D492A4604F12A
:101C50000800FFF729FF05F1CA0204F11000094945
:101C6000FFF722FF05F5CA7204F118000649BDE826
:101C70003840FFF719BF00BF902E00200824002035
:101C8000503400086134000828340008BFF34F8F37
:101C9000024AD368DB03FCD4704700BF003C02401B
:101CA00008B5094B1B7873B9FFF7F0FF074B1A69AA
:101CB000002ABFBF064A5A6002F188325A601A6889
:101CC00022F480621A6008BDEE300020003C024021
:101CD0002301674508B50B4B1B7893B9FFF7D6FF77
:101CE000094B1A6942F000421A611A6842F48052A4
:101CF0001A601A6822F480521A601A6842F48062EC
:101D00001A6008BDEE300020003C02400B2870B580
:101D100013D80B4A0B4C137863B90B4E4FF000618C
:101D200044F8231056F8235001330C2B2944F7D1E3
:101D30000123137054F8200070BD002070BD00BF57
:101D400020310020F0300020E8340008014B53F827
:101D500020007047E83400080C2070470B2810B5AD
:101D6000044601D9002010BDFFF7D0FF064B53F801
:101D700024301844C21A0BB9012010BD1268013278
:101D8000F0D1043BF6E700BFE83400080B2810B59B
:101D900004461ED8FFF77AFFFFF782FF0E49F323B0
:101DA000CB60FFF773FFC300DBB243F4007343F073
:101DB00002030B610B6943F480330B61FFF766FF8D
:101DC000FFF7A4FFFFF786FF2046BDE81040FFF7AE
:101DD000C5BF002010BD00BF003C02402DE9F84304
:101DE00012F00103154643D10244B2F1016F3FD214
:101DF0002C4B1B6813F001033AD02B4CFFF750FF1C
:101E0000F323E360FFF742FF40F20127032D16D8CA
:101E1000254C0F46401A40F20118EB1B0B44012BD6
:101E200000EB0706236926D823F001032361FFF79F
:101E300051FF0120BDE8F883043D0430E6E7830745
:101E4000E6D1236923F44073236123693B43236173
:101E500051F8046B0660BFF34F8FFFF717FF03685D
:101E60009E42E9D0236923F001032361FFF732FF8B
:101E70000020BDE8F88323F440732361236943EA1B
:101E800008032361B94637F8023B3380BFF34F8F15
:101E9000FFF7FCFE3688B9F80030B6B2B342BCD0CA
:101EA000E0E700BF00380240003C0240084908B5A6
:101EB0000B7828B153B9FFF7F3FE01230B7008BD6F
:101EC00023B1BDE808400870FFF704BF08BD00BF9C
:101ED000EE300020014B53F820007047502800409E
:101EE0000A4B1A6F120407D41A6F42F400721A6771
:101EF0001A6F42F400421A67054A136843F480736C
:101F0000136000B2034B43F82010704700380240C2
:101F10000070004050280040014B1868704700BF17
:101F20005028004001460020FFF7DABF38B5094BC2
:101F30001B689B000CD5084B084D01221A70002429
:101F4000E0B2FFF7C7FF45F824000134082CF7D1B1
:101F500038BD00BF743802404431002024310020D5
:101F6000014B1878704700BF4431002070470000D3
:101F7000FEE70000084A094B09498B4204D3094A8D
:101F80000021934205D3704752F8040F43F8040B25
:101F9000F3E743F8041BF4E79436000838340020D4
:101FA0003834002038340020836D30B500229D681D
:101FB000446D11464FF0FF3004EB4213013295425D
:101FC000C3F80019C3F81019C3F80809C3F8001BB7
:101FD000C3F8101BC3F8080BEED24FF00113C4F87E
:101FE0001C3830BD890141F02001016103699B0665
:101FF000FCD4122000F0CABE204B03EB80022DE976
:10200000F047D2F80CE05D6DDEF81420461CD2F8E3
:1020100000C005EB063605EB4018516861450BD34F
:10202000D5F83428012303FA00F022EA0000C5F8AD
:1020300034081846BDE8F087BEF81040ACEB010349
:10204000A34228BF2346D8F81849A4B2B3EB840FA3
:1020500010D894681F46A4F1040959F804AFC6F8D3
:1020600000A0042F01D9043FF7E71C440B449460FF
:102070005360D2E70020BDE8F08700BF4831002060
:1020800010B5054C2046FFF78FF84FF0A04363656D
:10209000024BA36510BD00BF483100203C3500084D
:1020A0000378012B70B5054650D12A4B446D9842F8
:1020B0001BD1294B5A6B42F080025A635A6D42F091
:1020C00080025A655A6D5A6942F080025A615A6913
:1020D00022F080025A610E2143205B6900F0D6FB9A
:1020E0001E4BE3601E4BC4F800380023C4F8003ECA
:1020F000C02323606E6D4FF40413A3633369002B78
:10210000FCDA012333610C2000F040FE3369DB0769
:10211000FCD4122000F03AFE3369002BFCDA0026D2
:10212000A6602846FFF740FF6B68C4F81068DB68BC
:10213000C4F81468C4F81C684BB90A4BA3614FF08B
:10214000FF336361A36843F00103A36070BD064BD6
:10215000F4E700BF4831002000380240401400403E
:1021600003002002003C30C0083C30C0F8B5446D8C
:10217000054600212046FFF735FFA96D00234FF0EB
:1021800001128F68C4F834384FF00066C4F81C2878
:102190004FF0FF3004EB431201339F42C2F8006955
:1021A000C2F8006BC2F80809C2F8080BF2D20B683B
:1021B0006A6DEB65636210231361166916F01006F1
:1021C000FBD1122000F0E2FDD4F8003823F4FE63C6
:1021D000C4F80038A36943F4402343F01003A3611B
:1021E0000923C4F81038C4F814380A4BEB604FF0D8
:1021F000C043C4F8103B084BC4F8003BC4F8106956
:10220000C4F80039EB6D03F1100243F48013EA6562
:10221000A362F8BD1835000840800010426D90F8A8
:102220004E10D2F8003823F4FE6343EA0113C2F8DB
:10223000003870472DE9F0410EB200EB86080D46DC
:10224000D8F80C100F6807F00303022B50D0032BB3
:1022500050D03D4A3D4F012B18BF1746446D4FEA01
:10226000451E04EB0E030022C3F8102B8A6905F10A
:10227000100C002A40D04A8A05F158035B013A430A
:10228000E2500123D4F81C2803FA0CF31343A644AC
:102290004A69C4F81C380023CEF8103905F13F0311
:1022A000002A39D00A8A898B9208012988BF4A43BB
:1022B000C16D04EB8303561841EA0242C665294604
:1022C0005A602046FFF78EFED8F80C301B8A43EA8E
:1022D00085531F4305F148035B01E7500123D4F800
:1022E0001C2803FA05F51543C4F81C58BDE8F08115
:1022F000174FB3E7174FB1E704EB4613D3F8002BA2
:1023000022F40042C3F8002BD4F81C28012303FA5E
:102310000CF322EA0303BAE704EB83030E4A5A6084
:1023200004EB461629462046FFF75CFED6F8003936
:1023300023F40043C6F80039D4F81C38012202FA0D
:1023400005F523EA0505CFE70080001000800410A2
:102350000080081000800C1000040002826D1268DA
:10236000C265FFF721BE00005831436D49015B583B
:1023700013F4004004D013F4001F14BF0120022006
:10238000704700004831436D49015B5813F4004029
:1023900004D013F4001F14BF012002207047000076
:1023A00000EB8101CB68196A0B6813604B685360BE
:1023B0007047000000EB810330B5DD68AA6913683F
:1023C000D36019B9402B84BF402313606B8A146813
:1023D000426D1C44013CB4FBF3F46343033323F02C
:1023E000030302EB411043EAC44343F0C043C0F887
:1023F000103B2B6803F00303012B09B20ED1D2F876
:10240000083802EB411013F4807FD0F8003B14BF72
:1024100043F0805343F00053C0F8003B02EB4112FD
:10242000D2F8003B43F00443C2F8003B30BD00004B
:102430002DE9F041244D6E6D06EB40130446D3F8B0
:10244000087BC3F8087B38070AD5D6F81438190773
:1024500006D505EB84032146DB6828465B68984770
:10246000FA072FD5D6F81438DB072BD505EB8403F4
:10247000D968CCB98B69488A5E68B6FBF0F200FB7C
:1024800012628AB91868DA6890420DD2121A83E88B
:102490001400202383F311880B482146FFF78AFF9D
:1024A00084F31188BDE8F081012303FA04F26B89FB
:1024B00023EA02036B81CB6823B121460248BDE8C1
:1024C000F0411847BDE8F0814831002000EB81035E
:1024D00070B5DD68436D6C692668E6604A0156BBDD
:1024E0001A444FF40020C2F810092A6802F00302CF
:1024F000012A0AB20ED1D3F8080803EB421410F4F3
:10250000807FD4F8000914BF40F0805040F00050A4
:10251000C4F8000903EB4212D2F8000940F004406D
:10252000C2F80009D3F83408012202FA01F101438C
:10253000C3F8341870BD19B9402E84BF4020206004
:1025400020682E8A841940F00050013C1A44B4FBE4
:10255000F6F440EAC440C6E7F8B504461E48456DA7
:1025600005EB4413D3F80869C3F80869F10717D5D8
:10257000D5F81038DA0713D500EB8403D9684B6916
:102580001F68DA68974218D2D21B00271A605F6072
:10259000202383F311882146FFF798FF87F31188E2
:1025A000330617D5D5F834280123A340134211D0A0
:1025B0002046BDE8F840FFF71FBD012303FA04F2EF
:1025C000038923EA020303818B68002BE8D02146AC
:1025D0009847E5E7F8BD00BF4831002096482DE94F
:1025E000F84F456D6E69AB691E4016F4805F6E61F1
:1025F000044605D0FEF744FEBDE8F84F00F05ABC93
:10260000002E12DAD5F8003E8B489B071EBFD5F886
:10261000003E23F00303C5F8003ED5F8043823F04C
:102620000103C5F80438FEF755FE370502D5824888
:10263000FEF744FEB0040CD5D5F8083813F0060FA9
:10264000EB6823F470530CBF43F4105343F4A053CE
:10265000EB60310704D56368DB680BB176489847B7
:10266000F2025AD4B3020CD5D4F85480DFF8C8A1D2
:1026700000274FF00109A36D9B68F9B28B4280F0EF
:102680008780F70619D5616D0A6AC2F30A1702F04E
:102690000F0302F4F012B2F5802F00F0A180B2F522
:1026A000402F0AD104EB830301F58051DB68186ADF
:1026B00000231A469F4240F087803003D5F818481F
:1026C00013D5E10302D50020FFF7B2FEA20302D525
:1026D0000120FFF7ADFE630302D50220FFF7A8FE3D
:1026E000270302D50320FFF7A3FE750384D5E00777
:1026F00002D50020FFF730FFA10702D50120FFF728
:102700002BFF620702D50220FFF726FF23077FF584
:1027100073AF0320FFF720FF6EE7D4F85480DFF893
:1027200018A100274FF00109A36D9B685FFA87FB92
:102730005B4597D308EB4B13D3F8002902F44022F2
:10274000B2F5802F22D1D3F80029002A1EDAD3F85F
:10275000002942F09042C3F80029D3F80029002A4A
:10276000FBDB5946606DFFF73DFC228909FA0BF34C
:1027700022EA0303238104EB8B03DB689B6813B11C
:102780005946504698475846FFF736FC0137CBE785
:1027900008EB4112D2F8003B03F44023B3F5802F3D
:1027A00010D1D2F8003B002B0CDA628909FA01F350
:1027B00022EA0303638104EB8103DB68DB680BB16E
:1027C00050469847013756E79C0708BF0A68072B11
:1027D00098BF027003F101039CBF120A013069E740
:1027E000023304EB830201F580515268906902685C
:1027F000D0F808C04068A2EB000E002210469742B5
:102800000AD104EB830463689B699A683A449A602E
:102810005A6817445F6050E712F0030F08BF08685A
:10282000964588BF8CF8000002F1010284BF000ABF
:102830000CF1010CE3E700BF48310020436D03EBCE
:102840004111D1F8003B43F40013C1F8003B70473D
:10285000436D03EB4111D1F8003943F40013C1F883
:1028600000397047436D03EB4111D1F8003B23F46D
:102870000013C1F8003B7047436D03EB4111D1F8E1
:10288000003923F40013C1F80039704700F16043A8
:1028900000F01F02400903F5614309018000C9B23D
:1028A00000F1604083F8001300F56140012393407C
:1028B000C0F880310360704730B5039C0172043367
:1028C00004FB0325C361049B03630021059B006097
:1028D0004060C1604261026185610462426281625E
:1028E000C162436330BD00000022416A4161016161
:1028F000C2608262C2626FF00101FFF70BB8000094
:1029000003694269934203D1C2680AB1002070474B
:10291000181D704703691960C2680132C260C2693C
:10292000134482690361934224BF436A0361002117
:10293000FEF7E4BF38B504460D46E3683BB1626973
:10294000131D1268A3621344E362002038BD237A8A
:1029500033B929462046FEF7C1FF0028EDDA38BD1D
:102960006FF00100FBE70000C368C269013BC36070
:102970004369134482694361934224BF436A4361BC
:1029800000238362036B03B11847704770B520239F
:10299000044683F31188866A3EB9FFF7CBFF0546EC
:1029A00018B186F31188284670BDA36AE26A13F84D
:1029B000015BA362934202D32046FFF7D5FF0023B9
:1029C00083F31188EFE700002DE9F84F04460E4627
:1029D00090469946202787F311880025AA46D4F807
:1029E00028B0BBF1000F09D149462046FFF7A2FFEE
:1029F00020B18BF311882846BDE8F88FA16AE36AFD
:102A0000A8EB050B5B1A9B4528BF9B46BBF1400F0B
:102A10001BD9334601F1400251F8040B43F8040B73
:102A20009142F9D1A36A40334036A3624035A26A8D
:102A3000E36A9A4202D32046FFF796FF8AF3118891
:102A40004545D8D287F31188C9E730465A46FEF784
:102A50009DF9A36A5B445E44A3625D44E7E700001E
:102A600010B5029C0172043303FB0421C3610023EF
:102A70008362C362039B0363049B00604060C46085
:102A800042610261816104624262436310BD0000E1
:102A9000026AC260426A4261026100228262C262CC
:102AA0006FF00101FEF736BF436902699A4203D114
:102AB000C2680AB100207047184650F8043B0B600A
:102AC00070470000C368C2690133C360436913449F
:102AD00082694361934224BF436A43610021FEF748
:102AE0000DBF000038B504460D46E3683BB12369CD
:102AF0001A1DA262E2691344E362002038BD237A02
:102B000033B929462046FEF7E9FE0028EDDA38BD44
:102B10006FF00100FBE7000003691960C268013A29
:102B2000C260C269134482690361934224BF436A4D
:102B3000036100238362036B03B1184770470000F1
:102B400070B5202304460E4683F31188856A35B993
:102B50001146FFF7C7FF10B185F3118870BDA36A56
:102B60001E70A36AE26A01339342A36204D3E1694F
:102B700020460439FFF7D0FF002080F3118870BD94
:102B80002DE9F84F04460D4691469A464FF020082D
:102B900088F311880026B346A76A4FB951462046EC
:102BA000FFF7A0FF20B187F311883046BDE8F88F0A
:102BB000A06AE76AA9EB06033F1A9F4228BF1F4697
:102BC000402F1BD905F1400355F8042B40F8042B86
:102BD0009D42F9D1A36A4033A3624036A26AE36AF8
:102BE0009A4204D3E16920460439FFF795FF8BF33D
:102BF00011884E45D9D288F31188CDE729463A4647
:102C0000FEF7C4F8A36A3B443D44A3623E44E5E7B3
:102C1000026943699A4203D1C3681BB918467047D9
:102C20000023FBE7836A002BF8D0043B9B1AF5D006
:102C30001360C368013BC360C3691A4483690261BE
:102C40009A4224BF436A0361002383620123E5E7BC
:102C500000F072B9034B002258631A610222DA6055
:102C6000704700BF000C0040014B0022DA60704743
:102C7000000C0040014B5863704700BF000C00403F
:102C8000FEE7000010B5174CFEF72EFDFEF750FED4
:102C9000802215492046FEF7D5FD012344F8180C83
:102CA0000374124B124AD96821F4E0610904090C3B
:102CB0000A431049DA60CA6842F08072CA600E495D
:102CC0000A6842F001020A601022DA77202283F8B3
:102CD0002220002383F3118862B60848BDE8104023
:102CE000FEF7D2BDB02900204835000800ED00E015
:102CF0000003FA05F0ED00E0001000E05035000898
:102D00002DE9F84F1F4CDFF88090656904F1140736
:102D10004FF00008D9F82430266AAA689E1B964214
:102D20001DD34FF0200AAA68236AD5F80CB01344CB
:102D300023622B68BB425F60A6EB02066361C5F8A5
:102D40000C8001D1FFF790FF88F311882869D847DC
:102D50008AF311886569AB689E42E4D2DAE762695A
:102D6000BA420CD0916823628E1B9660A868022834
:102D70002CBF1818981CBDE8F84FFFF77BBFBDE8C3
:102D8000F88F00BF88290020000C0040034B5968D1
:102D90005A68521A9042FBD8704700BF001000E0FA
:102DA0004B6843608B688360CB68C3600B69436189
:102DB0004B6903628B6943620B68036070470000D4
:102DC00008B5224B22481A6940F2FF110A431A61E2
:102DD0001A6922F4FF7222F001021A611A691A6B51
:102DE0000A431A631A6D0A431A651A4A1B6D114683
:102DF000FFF7D6FF184802F11C01FFF7D1FF174873
:102E000002F13801FFF7CCFF154802F15401FFF73A
:102E1000C7FF144802F17001FFF7C2FF124802F128
:102E20008C01FFF7BDFF114802F1A801FFF7B8FFC1
:102E30000F4802F1C401FFF7B3FF0E4802F1E001B1
:102E4000FFF7AEFFBDE8084000F0E2B800380240EE
:102E500000000240703500080004024000080240F3
:102E6000000C024000100240001402400018024012
:102E7000001C02400020024008B500F039FAFFF7BC
:102E800001FFFFF753F8BDE80840FEF7DBBE000086
:102E900070470000064A536823F001035360EFF3C4
:102EA0000983683383F30988002383F3118870470B
:102EB00030EF00E010B5202383F31188104B5B68DE
:102EC00013F4006318D0F1EE103AEFF309844FF0D9
:102ED000807344F84C3C0B4BDB6844F8083CA4F18D
:102EE000680383F30988FEF78DFC18B1064B44F89C
:102EF000503C10BD054BFAE783F3118810BD00BFAD
:102F000000ED00E030EF00E031030008340300087A
:102F1000084B1A69920710B508D500241C612023BC
:102F200083F31188FFF7ECFE84F31188BDE81040AD
:102F3000FFF7C0BF000C0040104B1A6C42F00802B3
:102F40001A641A6E42F008021A660D4A1B6E9368E4
:102F500043F0080393600B4B53229A624FF0FF3209
:102F6000DA6200229A615A63DA605A6001225A6179
:102F700008211A603220FFF789BC00BF00380240E8
:102F8000002004E0000C00401F4B1A696FEAC25297
:102F90006FEAD2521A611A69C2F308021A614FF03D
:102FA000FF301A695A69586100215A6959615A6992
:102FB0001A6A62F080521A621A6A02F080521A6229
:102FC0001A6A5A6A58625A6A59625A6A1A6C42F004
:102FD00080521A641A6E42F080521A661A6E0B4AB8
:102FE000106840F480701060186F00F44070B0F505
:102FF000007F1EBF4FF4803018671967536823F4B1
:103000000073536000F054B9003802400070004073
:10301000304B4FF080521A642F4A4FF440411160F8
:103020001A6842F001021A601A689207FCD59A6881
:1030300022F003029A60274B19469A6812F00C029C
:10304000FBD1186800F0F90018609A601A6842F421
:1030500080321A600B689B03FCD54B6F43F0010371
:103060004B671C4B5A6F9007FCD51C4A5A601A6874
:1030700042F080721A60184A53685904FCD5154B07
:103080001A689201FCD5164A9A60164B1A68164BBC
:103090009A42164B1BD1164A1168164A914216D114
:1030A00040F205121A600B4B9A6842F002029A60D5
:1030B0009A6802F00C02082AFAD15A6C42F4804253
:1030C0005A645A6E42F480425A665B6E704740F210
:1030D0000572E7E7003802400070004008544007DE
:1030E00000948838002004E011640020003C024075
:1030F00000ED00E041C20F41084A08B5536911686C
:103100000B4003F00103536123B1054A13680BB16F
:1031100050689847BDE80840FFF7CCBE003C01402E
:10312000B8330020084A08B5536911680B4003F012
:103130000203536123B1054A93680BB1D0689847E5
:10314000BDE80840FFF7B6BE003C0140B8330020A0
:10315000084A08B5536911680B4003F00403536132
:1031600023B1054A13690BB150699847BDE808407F
:10317000FFF7A0BE003C0140B8330020084A08B564
:10318000536911680B4003F00803536123B1054AEA
:1031900093690BB1D0699847BDE80840FFF78ABE34
:1031A000003C0140B8330020084A08B55369116853
:1031B0000B4003F01003536123B1054A136A0BB1AE
:1031C000506A9847BDE80840FFF774BE003C0140D4
:1031D000B8330020174B10B55C691A68144004F42A
:1031E00078725A61A30604D5134A936A0BB1D06A68
:1031F0009847600604D5104A136B0BB1506B984783
:10320000210604D50C4A936B0BB1D06B9847E205AD
:1032100004D5094A136C0BB1506C9847A30504D52B
:10322000054A936C0BB1D06C9847BDE81040FFF78E
:1032300041BE00BF003C0140B83300201A4B10B51E
:103240005C691A68144004F47C425A61620504D532
:10325000164A136D0BB1506D9847230504D5134AD8
:10326000936D0BB1D06D9847E00404D50F4A136EEF
:103270000BB1506E9847A10404D50C4A936E0BB164
:10328000D06E9847620404D5084A136F0BB1506F93
:103290009847230404D5054A936F0BB1D06F984724
:1032A000BDE81040FFF706BE003C0140B8330020E7
:1032B000062108B50846FFF7E9FA06210720FFF7BF
:1032C000E5FA06210820FFF7E1FA06210920FFF7B9
:1032D000DDFA06210A20FFF7D9FA06211720FFF7A9
:1032E000D5FA06212820BDE80840FFF7CFBA000034
:1032F00008B5FFF749FE00F00BF8FDF753FFFDF7A7
:1033000027FEFFF7C5FDBDE80840FFF7A1BC0000A0
:10331000002304491A465A50C8180833802B4260CB
:10332000F9D17047B8330020034611F8012B03F898
:10333000012B002AF9D1704712101213121100004C
:1033400053544D3332463F3F3F0000000000000021
:10335000403300083F000000130400007C330008E5
:103360003F00000019040000863300083F00000001
:1033700021040000903300083F00000053544D33F7
:1033800032463430780053544D333246343278006C
:1033900053544D3332463434365858000000000040
:1033A000C90E0008B50E0008F10E0008DD0E000879
:1033B000E90E0008D50E0008C10E0008AD0E000889
:1033C0004D0F000800000000010000000000000098
:1033D0000200000000000000F51000085D11000868
:1033E00040004000602E0020702E002002000000EF
:1033F000000000000300000000000000A111000810
:103400000000000010000000802E002000000000DE
:10341000010000000000000048310020010102000E
:1034200025424F41524425002553455249414C25E0
:10343000005652427261696E2D763531003031325C
:10344000333435363738394142434445460000006D
:103450004C61736572204E617669676174696F6E45
:103460000025424F415244252D424C00E51B0008E7
:103470004D1A000861100008C91B00084300000035
:103480008434000809024300020100C0320904002C
:1034900000010202010005240010010524010001C1
:1034A000042402020524060001070582030800FF28
:1034B00009040100020A00000007050102400000A3
:1034C000070581024000000012000000D03400080F
:1034D0001201100102000040AC275111000201024C
:1034E0000301000004030904004000000040000044
:1034F0000040000000400000000001000000020049
:1035000000000200000002000000020000000200B3
:10351000000002000000020000000000E9120008A4
:10352000C91500087516000840004000A8310020A9
:10353000A831002001000000B83100208000000008
:1035400040010000030000006D61696E0000000092
:1035500068350008C0310020B833002001000000A9
:10356000812C00080000000069646C650000000008
:103570000000802A00000000AAAAAAAA00000000F9
:10358000FFFF00000000000000A00A000000000093
:1035900000000000AAAAAAAA00000000FFFF000085
:1035A0000000000000000000000400000000000017
:1035B000AAAAAAAA00000000FFFF00000000000065
:1035C000000000000000001000000000AAAAAAAA43
:1035D00000000000FFFF00000000000000000000ED
:1035E0000000000000000000AAAAAAAA0000000033
:1035F000FFFF0000000000000000000000000000CD
:1036000000000000AAAAAAAA00000000FFFF000014
:1036100000000000000000000000000000000000AA
:10362000AAAAAAAA00000000FFFF000000000000F4
:103630000000000000000000000000000A00000080
:103640000000000003000000000000000000000077
:10365000000000000000000000000000000000006A
:10366000000000000000000000000000000000005A
:10367000FF0096000000000804000000E434000889
:10368000000000000000000000000000000000003A
:08369000000000000000000032
:00000001FF
